:02000000FE28D8
:10000800F000030E83120313A0000A08A1008A015E
:100018000B1DD728851DB3280A303B020318B328C7
:100028009C303402031C8328B608031D8328BC0AAD
:100038009B303402BE003C083E0203188328350872
:1000480003193628013A03194228033A03194E289E
:10005800013A03195A28073A03196628013A03197D
:1000680072287D28831203132E0A03193D28AE0A2D
:100078008028013083120313B500802883120313EC
:10008800AD0803194928AD038028023083120313F1
:10009800B5008028831203132F0A03195528AF0AC5
:1000A8008028033083120313B500802883120313BA
:1000B800AE0803196128AE038028043083120313A5
:1000C800B5008028831203132D0A03196D28AD0A81
:1000D8008028053083120313B50080288312031388
:1000E800AF0803197928AF03802883120313B501D9
:1000F800802883120313B50183120313BC0138301F
:10010800831203133402031CB3289C3034020318EF
:10011800B328B608031DB328BD0AC9303D02031C25
:10012800A328C00A37303402BF0040083F02031832
:10013800A028C0010130A40683120313BD01831255
:1001480003132418AB28AD01AE01AF01B328831205
:1001580003133708AD003808AE003908AF00831222
:100168000313B10A2D0831020318BC288614BF28CE
:10017800831203138610831203132E083102031807
:10018800C7288615CA2883120313861183120313FE
:100198002F0831020318D2280616D5288312031314
:1001A8000612CA220B11831203130C1CF528E9222C
:1001B800831203130C108519E828FF30AD00FF30B7
:1001C800AE00FF30AF00F5280A30831203133B025C
:1001D800031CF228AD01AE01AF01F5288312031309
:1001E800BB0A8312031321088A00200E8300F00E35
:1001F800700E0900982283120313A901AA010511A0
:100208000000861000008611000006120000AD01F3
:10021800AE01AF01BB01A410B501BF01BE01BC0115
:10022800C0012410B401262383120313A501A601DB
:100238000130112383120313A500A6012508A60087
:10024800A5010030112383120313A5070318A60A7A
:100258002508260403193A2901302602031C3F29E0
:10026800031D3A29FE302502031C3F290130831261
:100278000313A500A601262383120313861426233D
:100288008312031386100000861526238312031396
:100298008611000006162623831203130612000097
:1002A8008614000086150000061626238312031301
:1002B800861000008611000006122623C622E122BD
:1002C800831203138C1E6A291A08B00083120313C1
:1002D800181D7B29181218161A08B0001A08B00041
:1002E8001A08B000A901AA01BB01051588298312C3
:1002F8000313981C6429181218161A08B0001A0853
:10030800B0001A08B0006429831203138C1E8829D0
:10031800831203131A08B600A90A0319AA0A0511B9
:10032800B608031D0D2A0230831203132A02031C88
:10033800A229031DFC29A908031DFC298312031304
:100348001819FC29831203138C1EA6298312031380
:1003580029082506031DB7292A082606031DB729DB
:100368001A08B700F629831203132608A800250ADD
:10037800A7000319A80A29082706031DCA292A085D
:100388002806031DCA291A08B800F6298312031380
:100398002608A80002302507A7000318A80A29087C
:1003A8002706031DDE292A082806031DDE291A0848
:1003B800B900F629831203132608A800033025077D
:1003C800A7000318A80A29082706031DF2292A08E6
:1003D8002806031DF2291A08BA00F6298312031306
:1003E8001A08B00083120313A90A0319AA0A972945
:1003F80083120313851D622A3A08B4009C30340224
:100408000318622A3708AD003808AE003908AF0073
:10041800622A831203133608533A031D5E2A831295
:1004280003132A08031D622A053029020318622AC9
:100438001819622A831203138C1E1E2A83120313AF
:1004480029032A04031D2A2A1A08B7008312031352
:100458002908023A031D352AAA08031D352A1A0855
:10046800B800831203132908033A031D402AAA0877
:10047800031D402A1A08B900831203132908043AF5
:10048800031D582AAA08031D582A1A08BA00370853
:10049800413A031D582A3808543A031D582A390886
:1004A800B2003A08B300A41483120313A90A03196B
:1004B800AA0A132A831203131A08B000831203131B
:1004C800A41C6429A2013208F1220130831203130B
:1004D800A2003308F12283120313A501A6010130FB
:1004E800112383120313A500A6012508A600A50160
:1004F8000030112383120313A5070318A60AA410BA
:10050800250826040319922A01302602031C6429AF
:10051800031D922AFE302502031C64290130831230
:100528000313A500A601642983120313850186011C
:1005380083161C159C141C149B018B170B17E53094
:100548008600DB308500BC22CF22AA2A831603133B
:1005580018150430990018128312981798118316E9
:100568000C12181398128C128312181718160800F8
:100578008316031381128115CA220B118B120B17D4
:100588008B1708008B1608008B120800893083121D
:10059800031381000800831203139010901610169D
:1005A800901110108E010B308F00DB308E000C1074
:1005B80083160C140B178B170800831203131014DF
:1005C80008008312031310100800831203138E010E
:1005D8000B308F00DB308E00080083120313A3005A
:1005E8008B13831603178C130C158312031322081D
:1005F80003178D000313230803178C005530831647
:100608008D00AA308D008C14831603178C18082BC4
:10061800831603170C118B17080083120313A2000B
:10062800831603178C1383120313220803178D00F4
:1006380083160C14831603170C181E2B831203172A
:100648000C08080083120313A201A20104308312CC
:10065800031322020318452BAB01AC0183120313C9
:100668002C0F3A2BDC302B020318412B000083128D
:100678000313AB0A0319AC0A322B83120313A20A21
:040688002A2B080011
:02400E000A3F67
:00000001FF
